:100000000C9446000C9465000C9465000C946500FB
:100010000C9465000C9465000C9465000C946500CC
:100020000C9465000C9465000C9465000C946500BC
:100030000C9465000C9465000C9465000C946500AC
:100040000C9465000C9465000C9465000C9465009C
:100050000C9465000C9465000C9465000C9465008C
:100060000C9465000C9465000C9465000C9465007C
:100070000C9465000C9465000C9465000C9465006C
:100080000C9465000C9465000C94650011241FBE4F
:10009000CFEFD0E1DEBFCDBF11E0A0E0B1E0E2E5FF
:1000A000F1E000E00BBF02C007900D92A030B10755
:1000B000D9F711E0A0E0B1E001C01D92A030B10776
:1000C000E1F70E9467000C94A8000C940000CF9305
:1000D000DF93CDB7DEB721970FB6F894DEBF0FBE22
:1000E000CDBF1982E8E3F0E080E88083E2E3F0E04E
:1000F0001082E7E3F0E080E88083E1E3F0E0108243
:10010000E9E2F0E080E48083AAE2B0E0EAE2F0E035
:10011000808188618C9300C0EBE2F0E080818823CD
:100120002CF4ECE2F0E08081898301C0198289819E
:10013000882391F3EBE2F0E0808199278072907040
:100140000097C1F3ECE2F0E089818F5F8083E4CF18
:02015000FFCFDF
:00000001FF
